:02000000A12934
:08000800A1298207C034F9347C
:10001000A434B034993492348234F8348034903437
:1000200087348207D534E934FD3411342934573408
:1000300025343934613461346F3482076234623478
:1000400062346334633463346334633463346334F9
:100050006334100882070800342839283D284128D5
:1000600046284B284F285328170893004C21900A04
:100070000800C4305921900A080000305921900A24
:100080000800130811205921900A080013081D20A8
:100090005921900A080064305921900A0800003064
:1000A0005921900A08007421900117081302031DBA
:1000B000900A08001508820708007028602879282F
:1000C000851D69281E081902031D080001309500CE
:1000D00008004121D33019079E0003309500080025
:1000E000892183219A21383019079E00023095001A
:1000F000080085197F28D33019079E0008001E08C4
:100100001902031D08002B210130950008000D087D
:100110008207A728AA28B128B128AE28B128B1287B
:10012000AE28B128B128AE28B128B128AE28B12810
:10013000B128AE28B128B128AE28B128B128AE2800
:10014000B128B128AE28B128B128B3280800051D70
:100150008D0A0800051DB1288D010800051D031436
:100160008E0C8D0A0800051DBA2894140E098F0004
:100170008D0108000C158D010800140894108207E9
:1001800008000800C428D1280F08DF39463A0319AF
:10019000CF28153A031D0800942194010800940A01
:1001A000080030300F02031CCD28093C031CCD2869
:1001B00030300F029700950183219A2194010800A5
:1001C0000C080C1182070800FC280E29A129EB2835
:1001D000F8280A29A12995018921202183219A2122
:1001E000B43018079C000E3019079D008C0A0800D7
:1001F000B43018079C0000291C08180203190829AC
:100200001D081902031D08002B2194218C0A0800E7
:100210008C010800B43018079C0008001C08180264
:1002200003198C0108001A081802031D08001B0896
:100230001902031D0800960108001608850608002B
:100240002B3018079A0000300318013E19079B0055
:10025000103096000800A53018079A0004300318E3
:10026000013E19079B001030960008001530180752
:100270009A000E300318013E19079B0010309600BB
:1002800008002B3018079A001C300318013E19078C
:100290009B001030960008000C30831685008312F6
:1002A00085140000051400008510000005100000F2
:1002B000080092000C3083168500831208309100EC
:1002C000920D8514031C8510000005140000051014
:1002D0000000910B60290E308316850083120514EF
:1002E00000000510000008000C3083168500831202
:1002F0008510000005140000851400000F308316DF
:100300008500831208009008031D0800013090004A
:100310000800970A01301702031C9129043C0318B6
:1003200008000130970008009508031D08000130FF
:10033000950008001708052086009508031D861300
:10034000080083168601EF308500C13081008312DA
:100350008601950194018C018D019001960199010E
:1003600098013621051DC929053097008321942164
:1003700096080319D0290B1DBB29BC3081000B1135
:1003800064001D2129201321980A031DB829990A08
:10039000B8290A3097009A2183211D308D00D02979
:1003A0000B1DD029BC3081000B1164001D2187205A
:1003B00029205A20E020BD201321980A031DD029AE
:0403C000990AD0299D
:02400E00FD3F74
:00000001FF
